 gpiosdk

 Timestamp is 4da2a539 (Mon Apr 11 18:52:41 2011)

 Preferred load address is 10000000

 Start         Length     Name                   Class
 0001:00000000 00000004H .CRT$XCA                CODE
 0001:00000004 00000004H .CRT$XCZ                CODE
 0001:00000008 00000004H .CRT$XIA                CODE
 0001:0000000c 00000004H .CRT$XIZ                CODE
 0001:00000010 00000004H .CRT$XPA                CODE
 0001:00000014 00000004H .CRT$XPZ                CODE
 0001:00000018 00000004H .CRT$XTA                CODE
 0001:0000001c 00000004H .CRT$XTZ                CODE
 0001:00000020 00000fb8H .rdata                  CODE
 0001:00000fd8 00000024H .rdata$debug            CODE
 0001:00000ffc 00001ca4H .text                   CODE
 0001:00002ca0 00000014H .xdata                  CODE
 0001:00002cb4 00000014H .idata$2                CODE
 0001:00002cc8 00000014H .idata$3                CODE
 0001:00002cdc 00000048H .idata$4                CODE
 0001:00002d24 0000000cH .idata$6                CODE
 0001:00002d30 000001a5H .edata                  CODE
 0002:00000000 00000048H .idata$5                DATA
 0002:00000048 00000450H .data                   DATA
 0002:00000498 00000fb4H .bss                    DATA
 0003:00000000 00000118H .pdata                  DATA

  Address         Publics by Value              Rva+Base       Lib:Object

 0000:00000000       ___safe_se_handler_count   00000000     <absolute>
 0000:00000000       ___safe_se_handler_table   00000000     <absolute>
 0001:00000000       __xc_a                     10001000     corelib0:crt0init.obj
 0001:00000004       __xc_z                     10001004     corelib0:crt0init.obj
 0001:00000008       __xi_a                     10001008     corelib0:crt0init.obj
 0001:0000000c       __xi_z                     1000100c     corelib0:crt0init.obj
 0001:00000010       __xp_a                     10001010     corelib0:crt0init.obj
 0001:00000014       __xp_z                     10001014     corelib0:crt0init.obj
 0001:00000018       __xt_a                     10001018     corelib0:crt0init.obj
 0001:0000001c       __xt_z                     1000101c     corelib0:crt0init.obj
 0001:0000003c       ??_C@_1DG@HDKGPHBH@?$AAG?$AAP?$AAI?$AAO?$AA?5?$AAS?$AAD?$AAK?$AA?3?$AA?5?$AA?9?$AAG?$AAp?$AAi?$AAo?$AAI?$AAn?$AAi?$AAt?$AA?$CI?$AA?$CF?$AAs?$AA?$CJ?$AA?9?$AA?$AN?$AA?6?$AA?$AA@ 1000103c     gpiosdk.obj
 0001:00000074       ??_C@_1M@HCOOECOK@?$AAF?$AAA?$AAL?$AAS?$AAE?$AA?$AA@ 10001074     gpiosdk.obj
 0001:00000080       ??_C@_19ELAAHEEL@?$AAT?$AAR?$AAU?$AAE?$AA?$AA@ 10001080     gpiosdk.obj
 0001:00000090       ??_C@_1IA@KDMGMEFO@?$AAG?$AAP?$AAI?$AAO?$AA?5?$AAS?$AAD?$AAK?$AA?3?$AA?5?$AA?5?$AAG?$AAp?$AAi?$AAo?$AAI?$AAn?$AAi?$AAt?$AA?$DO?$AA?5?$AAW?$AAA?$AAR?$AAN?$AAI?$AAN?$AAG?$AA?3?$AA?5?$AAG?$AAp@ 10001090     gpiosdk.obj
 0001:00000110       ??_C@_1IA@HKPMIDEL@?$AAG?$AAP?$AAI?$AAO?$AA?5?$AAS?$AAD?$AAK?$AA?3?$AA?5?$AA?5?$AAG?$AAp?$AAi?$AAo?$AAI?$AAn?$AAi?$AAt?$AA?$DO?$AA?5?$AAE?$AAR?$AAR?$AAO?$AAR?$AA?3?$AA?5?$AAC?$AAa?$AAn?$AA?8@ 10001110     gpiosdk.obj
 0001:00000190       ??_C@_1KE@GPLAMEHD@?$AAG?$AAP?$AAI?$AAO?$AA?5?$AAS?$AAD?$AAK?$AA?3?$AA?5?$AA?5?$AAG?$AAp?$AAi?$AAo?$AAI?$AAn?$AAi?$AAt?$AA?$DO?$AA?5?$AAI?$AAN?$AAF?$AAO?$AA?3?$AA?5?$AAC?$AAo?$AAn?$AAn?$AAe@ 10001190     gpiosdk.obj
 0001:00000234       ??_C@_1M@BPKHPEKM@?$AAG?$AAP?$AAI?$AA1?$AA?3?$AA?$AA@ 10001234     gpiosdk.obj
 0001:00000240       ??_C@_1DC@PMFODJCI@?$AAG?$AAP?$AAI?$AAO?$AA?5?$AAS?$AAD?$AAK?$AA?3?$AA?5?$AA?$CL?$AAG?$AAp?$AAi?$AAo?$AAI?$AAn?$AAi?$AAt?$AA?$CI?$AA?$CJ?$AA?$CL?$AA?$AN?$AA?6?$AA?$AA@ 10001240     gpiosdk.obj
 0001:00000274       ??_C@_1DK@PPLLHEOO@?$AAG?$AAP?$AAI?$AAO?$AA?5?$AAS?$AAD?$AAK?$AA?3?$AA?5?$AA?9?$AAG?$AAp?$AAi?$AAo?$AAD?$AAe?$AAi?$AAn?$AAi?$AAt?$AA?$CI?$AA?$CF?$AAs?$AA?$CJ?$AA?9?$AA?$AN?$AA?6?$AA?$AA@ 10001274     gpiosdk.obj
 0001:000002b0       ??_C@_1II@FEOCKJLO@?$AAG?$AAP?$AAI?$AAO?$AA?5?$AAS?$AAD?$AAK?$AA?3?$AA?5?$AA?5?$AAG?$AAp?$AAi?$AAo?$AAD?$AAe?$AAi?$AAn?$AAi?$AAt?$AA?$DO?$AA?5?$AAW?$AAA?$AAR?$AAN?$AAI?$AAN?$AAG?$AA?3?$AA?5@ 100012b0     gpiosdk.obj
 0001:00000338       ??_C@_1IG@FPOAIHJB@?$AAG?$AAP?$AAI?$AAO?$AA?5?$AAS?$AAD?$AAK?$AA?3?$AA?5?$AA?5?$AAG?$AAp?$AAi?$AAo?$AAD?$AAe?$AAi?$AAn?$AAi?$AAt?$AA?$DO?$AA?5?$AAE?$AAR?$AAR?$AAO?$AAR?$AA?3?$AA?5?$AAC?$AAa@ 10001338     gpiosdk.obj
 0001:000003c0       ??_C@_1IC@ODPCKDFD@?$AAG?$AAP?$AAI?$AAO?$AA?5?$AAS?$AAD?$AAK?$AA?3?$AA?5?$AA?5?$AAG?$AAp?$AAi?$AAo?$AAD?$AAe?$AAi?$AAn?$AAi?$AAt?$AA?$DO?$AA?5?$AAI?$AAN?$AAF?$AAO?$AA?3?$AA?5?$AAC?$AAl?$AAo@ 100013c0     gpiosdk.obj
 0001:00000444       ??_C@_1DG@JPAMHOLH@?$AAG?$AAP?$AAI?$AAO?$AA?5?$AAS?$AAD?$AAK?$AA?3?$AA?5?$AA?$CL?$AAG?$AAp?$AAi?$AAo?$AAD?$AAe?$AAi?$AAn?$AAi?$AAt?$AA?$CI?$AA?$CJ?$AA?$CL?$AA?$AN?$AA?6?$AA?$AA@ 10001444     gpiosdk.obj
 0001:00000480       ??_C@_1EA@EMLAMHOB@?$AAG?$AAP?$AAI?$AAO?$AA?5?$AAS?$AAD?$AAK?$AA?3?$AA?5?$AA?9?$AAG?$AAp?$AAi?$AAo?$AAG?$AAe?$AAt?$AAC?$AAo?$AAn?$AAf?$AAi?$AAg?$AA?$CI?$AA?$CF?$AAs?$AA?$CJ?$AA?9?$AA?$AN?$AA?6?$AA?$AA@ 10001480     gpiosdk.obj
 0001:000004c0       ??_C@_1GE@FNIFMANG@?$AAG?$AAP?$AAI?$AAO?$AA?5?$AAS?$AAD?$AAK?$AA?3?$AA?5?$AA?$CL?$AAG?$AAp?$AAi?$AAo?$AAG?$AAe?$AAt?$AAC?$AAo?$AAn?$AAf?$AAi?$AAg?$AA?$CI?$AAp?$AAG?$AAp?$AAi?$AAo?$AAC?$AAo@ 100014c0     gpiosdk.obj
 0001:00000524       ??_C@_1DK@LNEBJDAF@?$AAG?$AAP?$AAI?$AAO?$AA?5?$AAS?$AAD?$AAK?$AA?3?$AA?5?$AA?9?$AAC?$AAa?$AAl?$AAl?$AAD?$AAr?$AAi?$AAv?$AAe?$AAr?$AA?$CI?$AA?$CF?$AAs?$AA?$CJ?$AA?9?$AA?$AN?$AA?6?$AA?$AA@ 10001524     gpiosdk.obj
 0001:00000560       ??_C@_1KC@ICFOHGEE@?$AAG?$AAP?$AAI?$AAO?$AA?5?$AAS?$AAD?$AAK?$AA?3?$AA?5?$AA?5?$AAC?$AAa?$AAl?$AAl?$AAD?$AAr?$AAi?$AAv?$AAe?$AAr?$AA?$DO?$AA?5?$AAE?$AAR?$AAR?$AAO?$AAR?$AA?3?$AA?5?$AAG?$AAP@ 10001560     gpiosdk.obj
 0001:00000608       ??_C@_1IE@HHNJFJFH@?$AAG?$AAP?$AAI?$AAO?$AA?5?$AAS?$AAD?$AAK?$AA?3?$AA?5?$AA?5?$AAC?$AAa?$AAl?$AAl?$AAD?$AAr?$AAi?$AAv?$AAe?$AAr?$AA?$DO?$AA?5?$AAW?$AAA?$AAR?$AAN?$AAI?$AAN?$AAG?$AA?3?$AA?5@ 10001608     gpiosdk.obj
 0001:00000690       ??_C@_1IG@FCNIBJFD@?$AAG?$AAP?$AAI?$AAO?$AA?5?$AAS?$AAD?$AAK?$AA?3?$AA?5?$AA?$CL?$AAC?$AAa?$AAl?$AAl?$AAD?$AAr?$AAi?$AAv?$AAe?$AAr?$AA?$CI?$AAI?$AAo?$AAc?$AAt?$AAl?$AAC?$AAo?$AAd?$AAe?$AA?5@ 10001690     gpiosdk.obj
 0001:00000718       ??_C@_1EA@PLAPJKJK@?$AAG?$AAP?$AAI?$AAO?$AA?5?$AAS?$AAD?$AAK?$AA?3?$AA?5?$AA?9?$AAG?$AAp?$AAi?$AAo?$AAS?$AAe?$AAt?$AAC?$AAo?$AAn?$AAf?$AAi?$AAg?$AA?$CI?$AA?$CF?$AAs?$AA?$CJ?$AA?9?$AA?$AN?$AA?6?$AA?$AA@ 10001718     gpiosdk.obj
 0001:00000758       ??_C@_1GE@HFFILCEM@?$AAG?$AAP?$AAI?$AAO?$AA?5?$AAS?$AAD?$AAK?$AA?3?$AA?5?$AA?$CL?$AAG?$AAp?$AAi?$AAo?$AAS?$AAe?$AAt?$AAC?$AAo?$AAn?$AAf?$AAi?$AAg?$AA?$CI?$AAp?$AAG?$AAp?$AAi?$AAo?$AAC?$AAo@ 10001758     gpiosdk.obj
 0001:000007bc       ??_C@_1DM@NPKLKGAD@?$AAG?$AAP?$AAI?$AAO?$AA?5?$AAS?$AAD?$AAK?$AA?3?$AA?5?$AA?9?$AAG?$AAp?$AAi?$AAo?$AAR?$AAe?$AAa?$AAd?$AAP?$AAi?$AAn?$AA?$CI?$AA?$CF?$AAs?$AA?$CJ?$AA?9?$AA?$AN?$AA?6?$AA?$AA@ 100017bc     gpiosdk.obj
 0001:000007f8       ??_C@_1FE@HNELDGOI@?$AAG?$AAP?$AAI?$AAO?$AA?5?$AAS?$AAD?$AAK?$AA?3?$AA?5?$AA?$CL?$AAG?$AAp?$AAi?$AAo?$AAR?$AAe?$AAa?$AAd?$AAP?$AAi?$AAn?$AA?$CI?$AAp?$AAG?$AAp?$AAi?$AAo?$AA?5?$AA?$DN?$AA?5?$AA0@ 100017f8     gpiosdk.obj
 0001:00000850       ??_C@_1HK@NINCMAGM@?$AAG?$AAP?$AAI?$AAO?$AA?5?$AAS?$AAD?$AAK?$AA?3?$AA?5?$AA?$CL?$AAC?$AAa?$AAl?$AAl?$AAD?$AAr?$AAi?$AAv?$AAe?$AAr?$AA?$CI?$AAI?$AAo?$AAc?$AAt?$AAl?$AAC?$AAo?$AAd?$AAe?$AA?5@ 10001850     gpiosdk.obj
 0001:000008cc       ??_C@_1DO@MHDJFLHL@?$AAG?$AAP?$AAI?$AAO?$AA?5?$AAS?$AAD?$AAK?$AA?3?$AA?5?$AA?9?$AAG?$AAp?$AAi?$AAo?$AAW?$AAr?$AAi?$AAt?$AAe?$AAP?$AAi?$AAn?$AA?$CI?$AA?$CF?$AAs?$AA?$CJ?$AA?9?$AA?$AN?$AA?6?$AA?$AA@ 100018cc     gpiosdk.obj
 0001:00000910       ??_C@_1FG@MDHMAICK@?$AAG?$AAP?$AAI?$AAO?$AA?5?$AAS?$AAD?$AAK?$AA?3?$AA?5?$AA?$CL?$AAG?$AAp?$AAi?$AAo?$AAW?$AAr?$AAi?$AAt?$AAe?$AAP?$AAi?$AAn?$AA?$CI?$AAp?$AAG?$AAp?$AAi?$AAo?$AA?5?$AA?$DN?$AA?5@ 10001910     gpiosdk.obj
 0001:00000968       ??_C@_1DO@FPKEHBGG@?$AAG?$AAP?$AAI?$AAO?$AA?5?$AAS?$AAD?$AAK?$AA?3?$AA?5?$AA?9?$AAG?$AAp?$AAi?$AAo?$AAR?$AAe?$AAa?$AAd?$AAP?$AAo?$AAr?$AAt?$AA?$CI?$AA?$CF?$AAs?$AA?$CJ?$AA?9?$AA?$AN?$AA?6?$AA?$AA@ 10001968     gpiosdk.obj
 0001:000009a8       ??_C@_1FG@CBIGHAPB@?$AAG?$AAP?$AAI?$AAO?$AA?5?$AAS?$AAD?$AAK?$AA?3?$AA?5?$AA?$CL?$AAG?$AAp?$AAi?$AAo?$AAR?$AAe?$AAa?$AAd?$AAP?$AAo?$AAr?$AAt?$AA?$CI?$AAp?$AAG?$AAp?$AAi?$AAo?$AA?5?$AA?$DN?$AA?5@ 100019a8     gpiosdk.obj
 0001:00000a00       ??_C@_1EA@HLEOBEKL@?$AAG?$AAP?$AAI?$AAO?$AA?5?$AAS?$AAD?$AAK?$AA?3?$AA?5?$AA?9?$AAG?$AAp?$AAi?$AAo?$AAW?$AAr?$AAi?$AAt?$AAe?$AAP?$AAo?$AAr?$AAt?$AA?$CI?$AA?$CF?$AAs?$AA?$CJ?$AA?9?$AA?$AN?$AA?6?$AA?$AA@ 10001a00     gpiosdk.obj
 0001:00000a40       ??_C@_1FI@BJCLGGKB@?$AAG?$AAP?$AAI?$AAO?$AA?5?$AAS?$AAD?$AAK?$AA?3?$AA?5?$AA?$CL?$AAG?$AAp?$AAi?$AAo?$AAW?$AAr?$AAi?$AAt?$AAe?$AAP?$AAo?$AAr?$AAt?$AA?$CI?$AAp?$AAG?$AAp?$AAi?$AAo?$AA?5?$AA?$DN@ 10001a40     gpiosdk.obj
 0001:00000a98       ??_C@_1EE@GJIJEDPI@?$AAG?$AAP?$AAI?$AAO?$AA?5?$AAS?$AAD?$AAK?$AA?3?$AA?5?$AA?9?$AAG?$AAp?$AAi?$AAo?$AAR?$AAe?$AAa?$AAd?$AAI?$AAn?$AAt?$AAr?$AAP?$AAi?$AAn?$AA?$CI?$AA?$CF?$AAs?$AA?$CJ?$AA?9?$AA?$AN@ 10001a98     gpiosdk.obj
 0001:00000ae0       ??_C@_1FM@PCPMLBHN@?$AAG?$AAP?$AAI?$AAO?$AA?5?$AAS?$AAD?$AAK?$AA?3?$AA?5?$AA?$CL?$AAG?$AAp?$AAi?$AAo?$AAR?$AAe?$AAa?$AAd?$AAI?$AAn?$AAt?$AAr?$AAP?$AAi?$AAn?$AA?$CI?$AAp?$AAG?$AAp?$AAi?$AAo@ 10001ae0     gpiosdk.obj
 0001:00000b40       ??_C@_1EG@HIIMOJMF@?$AAG?$AAP?$AAI?$AAO?$AA?5?$AAS?$AAD?$AAK?$AA?3?$AA?5?$AA?9?$AAG?$AAp?$AAi?$AAo?$AAR?$AAe?$AAa?$AAd?$AAI?$AAn?$AAt?$AAr?$AAP?$AAo?$AAr?$AAt?$AA?$CI?$AA?$CF?$AAs?$AA?$CJ?$AA?9@ 10001b40     gpiosdk.obj
 0001:00000b88       ??_C@_1FO@FOGMJHJK@?$AAG?$AAP?$AAI?$AAO?$AA?5?$AAS?$AAD?$AAK?$AA?3?$AA?5?$AA?$CL?$AAG?$AAp?$AAi?$AAo?$AAR?$AAe?$AAa?$AAd?$AAI?$AAn?$AAt?$AAr?$AAP?$AAo?$AAr?$AAt?$AA?$CI?$AAp?$AAG?$AAp?$AAi@ 10001b88     gpiosdk.obj
 0001:00000be8       ??_C@_1EG@NAMPCJFD@?$AAG?$AAP?$AAI?$AAO?$AA?5?$AAS?$AAD?$AAK?$AA?3?$AA?5?$AA?9?$AAG?$AAp?$AAi?$AAo?$AAC?$AAl?$AAe?$AAa?$AAr?$AAI?$AAn?$AAt?$AAr?$AAP?$AAi?$AAn?$AA?$CI?$AA?$CF?$AAs?$AA?$CJ?$AA?9@ 10001be8     gpiosdk.obj
 0001:00000c30       ??_C@_1FO@KBGCFLEH@?$AAG?$AAP?$AAI?$AAO?$AA?5?$AAS?$AAD?$AAK?$AA?3?$AA?5?$AA?$CL?$AAG?$AAp?$AAi?$AAo?$AAC?$AAl?$AAe?$AAa?$AAr?$AAI?$AAn?$AAt?$AAr?$AAP?$AAi?$AAn?$AA?$CI?$AAp?$AAG?$AAp?$AAi@ 10001c30     gpiosdk.obj
 0001:00000c90       ??_C@_1EI@JIBILNOH@?$AAG?$AAP?$AAI?$AAO?$AA?5?$AAS?$AAD?$AAK?$AA?3?$AA?5?$AA?9?$AAG?$AAp?$AAi?$AAo?$AAC?$AAl?$AAe?$AAa?$AAr?$AAI?$AAn?$AAt?$AAr?$AAP?$AAo?$AAr?$AAt?$AA?$CI?$AA?$CF?$AAs?$AA?$CJ@ 10001c90     gpiosdk.obj
 0001:00000cd8       ??_C@_1GA@DLBKBBBL@?$AAG?$AAP?$AAI?$AAO?$AA?5?$AAS?$AAD?$AAK?$AA?3?$AA?5?$AA?$CL?$AAG?$AAp?$AAi?$AAo?$AAC?$AAl?$AAe?$AAa?$AAr?$AAI?$AAn?$AAt?$AAr?$AAP?$AAo?$AAr?$AAt?$AA?$CI?$AAp?$AAG?$AAp@ 10001cd8     gpiosdk.obj
 0001:00000d38       ??_C@_1EI@EBOKLGHB@?$AAG?$AAP?$AAI?$AAO?$AA?5?$AAS?$AAD?$AAK?$AA?3?$AA?5?$AA?9?$AAG?$AAp?$AAi?$AAo?$AAR?$AAe?$AAg?$AAi?$AAs?$AAt?$AAe?$AAr?$AAE?$AAv?$AAe?$AAn?$AAt?$AA?$CI?$AA?$CF?$AAs?$AA?$CJ@ 10001d38     gpiosdk.obj
 0001:00000d80       ??_C@_1GK@OHNGHPDN@?$AAG?$AAP?$AAI?$AAO?$AA?5?$AAS?$AAD?$AAK?$AA?3?$AA?5?$AA?$CL?$AAG?$AAp?$AAi?$AAo?$AAR?$AAe?$AAg?$AAi?$AAs?$AAt?$AAe?$AAr?$AAE?$AAv?$AAe?$AAn?$AAt?$AA?$CI?$AAp?$AAG?$AAp@ 10001d80     gpiosdk.obj
 0001:00000df0       ??_C@_1IE@FCLCEIOB@?$AAG?$AAP?$AAI?$AAO?$AA?5?$AAS?$AAD?$AAK?$AA?3?$AA?5?$AA?$CL?$AAC?$AAa?$AAl?$AAl?$AAD?$AAr?$AAi?$AAv?$AAe?$AAr?$AA?$CI?$AAI?$AAo?$AAc?$AAt?$AAl?$AAC?$AAo?$AAd?$AAe?$AA?5@ 10001df0     gpiosdk.obj
 0001:00000e78       ??_C@_1EM@NDODGJKB@?$AAG?$AAP?$AAI?$AAO?$AA?5?$AAS?$AAD?$AAK?$AA?3?$AA?5?$AA?9?$AAG?$AAp?$AAi?$AAo?$AAD?$AAe?$AAr?$AAe?$AAg?$AAi?$AAs?$AAt?$AAe?$AAr?$AAE?$AAv?$AAe?$AAn?$AAt?$AA?$CI?$AA?$CF@ 10001e78     gpiosdk.obj
 0001:00000ec8       ??_C@_1GO@PDNLPJB@?$AAG?$AAP?$AAI?$AAO?$AA?5?$AAS?$AAD?$AAK?$AA?3?$AA?5?$AA?$CL?$AAG?$AAp?$AAi?$AAo?$AAD?$AAe?$AAr?$AAe?$AAg?$AAi?$AAs?$AAt?$AAe?$AAr?$AAE?$AAv?$AAe?$AAn?$AAt?$AA?$CI?$AAp@ 10001ec8     gpiosdk.obj
 0001:00000f38       ??_C@_1DO@FMFABLPE@?$AAG?$AAP?$AAI?$AAO?$AA?5?$AAS?$AAD?$AAK?$AA?3?$AA?5?$AA?9?$AAG?$AAp?$AAi?$AAo?$AAG?$AAe?$AAt?$AAE?$AAv?$AAe?$AAn?$AAt?$AA?$CI?$AA?$CF?$AAs?$AA?$CJ?$AA?9?$AA?$AN?$AA?6?$AA?$AA@ 10001f38     gpiosdk.obj
 0001:00000f78       ??_C@_1GA@PGLEIGFL@?$AAG?$AAP?$AAI?$AAO?$AA?5?$AAS?$AAD?$AAK?$AA?3?$AA?5?$AA?$CL?$AAG?$AAp?$AAi?$AAo?$AAG?$AAe?$AAt?$AAE?$AAv?$AAe?$AAn?$AAt?$AA?$CI?$AAp?$AAG?$AAp?$AAi?$AAo?$AAE?$AAv?$AAe@ 10001f78     gpiosdk.obj
 0001:00000ffc       ?to_T@@YAPBGPBD@Z          10001ffc f   DebugZones.obj
 0001:00001098       DllMain                    10002098 f   gpiosdk.obj
 0001:000010e4       GpioInit                   100020e4 f   gpiosdk.obj
 0001:000012ec       GpioDeinit                 100022ec f   gpiosdk.obj
 0001:0000149c       GpioGetConfig              1000249c f   gpiosdk.obj
 0001:00001758       GpioSetConfig              10002758 f   gpiosdk.obj
 0001:00001834       GpioReadPin                10002834 f   gpiosdk.obj
 0001:00001abc       GpioWritePin               10002abc f   gpiosdk.obj
 0001:00001b98       GpioReadPort               10002b98 f   gpiosdk.obj
 0001:00001c74       GpioWritePort              10002c74 f   gpiosdk.obj
 0001:00001d50       GpioReadIntrPin            10002d50 f   gpiosdk.obj
 0001:00001e2c       GpioReadIntrPort           10002e2c f   gpiosdk.obj
 0001:00001f08       GpioClearIntrPin           10002f08 f   gpiosdk.obj
 0001:00001fe4       GpioClearIntrPort          10002fe4 f   gpiosdk.obj
 0001:000020c0       GpioRegisterEvent          100030c0 f   gpiosdk.obj
 0001:00002348       GpioDeregisterEvent        10003348 f   gpiosdk.obj
 0001:00002424       GpioGetEvent               10003424 f   gpiosdk.obj
 0001:00002500       RegisterDbgZones           10003500 f   coredll:COREDLL.dll
 0001:00002510       DisableThreadLibraryCalls  10003510 f   coredll:COREDLL.dll
 0001:00002520       GetLastError               10003520 f   coredll:COREDLL.dll
 0001:00002530       CreateFileW                10003530 f   coredll:COREDLL.dll
 0001:00002540       NKDbgPrintfW               10003540 f   coredll:COREDLL.dll
 0001:00002550       CloseHandle                10003550 f   coredll:COREDLL.dll
 0001:00002560       SetLastError               10003560 f   coredll:COREDLL.dll
 0001:00002570       DeviceIoControl            10003570 f   coredll:COREDLL.dll
 0001:00002580       _DllMainCRTStartup         10003580 f   corelib0:pegdmain.obj
 0001:00002718       __security_init_cookie     10003718 f   corelib0:seccinit.obj
 0001:000027b0       exit                       100037b0 f   corelib0:cexit.obj
 0001:000028d4       _exit                      100038d4 f   corelib0:cexit.obj
 0001:000028f4       _cexit                     100038f4 f   corelib0:cexit.obj
 0001:0000290c       _c_exit                    1000390c f   corelib0:cexit.obj
 0001:00002924       _initterm                  10003924 f   corelib0:crt0dat.obj
 0001:00002970       _cinit                     10003970 f   corelib0:crt0dat.obj
 0001:000029a0       __crt_ExitProcess          100039a0 f   corelib0:exitproc_proxy.obj
 0001:000029cc       GetCurrentProcess          100039cc f i corelib0:exitproc_proxy.obj
 0001:000029e4       _onexit                    100039e4 f   corelib0:onexit.obj
 0001:00002bc0       atexit                     10003bc0 f   corelib0:onexit.obj
 0001:00002c10       mbstowcs                   10003c10 f   corelib1:COREDLL.dll
 0001:00002c20       _XcptFilter                10003c20 f   corelib1:COREDLL.dll
 0001:00002c30       __C_specific_handler       10003c30 f   corelib1:COREDLL.dll
 0001:00002c40       __security_gen_cookie2     10003c40 f   corelib1:COREDLL.dll
 0001:00002c50       free                       10003c50 f   corelib1:COREDLL.dll
 0001:00002c60       realloc                    10003c60 f   corelib1:COREDLL.dll
 0001:00002c70       malloc                     10003c70 f   corelib1:COREDLL.dll
 0001:00002c80       _msize                     10003c80 f   corelib1:COREDLL.dll
 0001:00002c90       TerminateProcess           10003c90 f   coredll:COREDLL.dll
 0001:00002cb4       __IMPORT_DESCRIPTOR_COREDLL 10003cb4     coredll:COREDLL.dll
 0001:00002cc8       __NULL_IMPORT_DESCRIPTOR   10003cc8     coredll:COREDLL.dll
 0002:00000000       __imp_RegisterDbgZones     10004000     coredll:COREDLL.dll
 0002:00000004       __imp_DisableThreadLibraryCalls 10004004     coredll:COREDLL.dll
 0002:00000008       __imp_GetLastError         10004008     coredll:COREDLL.dll
 0002:0000000c       __imp_CreateFileW          1000400c     coredll:COREDLL.dll
 0002:00000010       __imp_NKDbgPrintfW         10004010     coredll:COREDLL.dll
 0002:00000014       __imp_CloseHandle          10004014     coredll:COREDLL.dll
 0002:00000018       __imp_SetLastError         10004018     coredll:COREDLL.dll
 0002:0000001c       __imp_DeviceIoControl      1000401c     coredll:COREDLL.dll
 0002:00000020       __imp_mbstowcs             10004020     corelib1:COREDLL.dll
 0002:00000024       __imp__XcptFilter          10004024     corelib1:COREDLL.dll
 0002:00000028       __imp___C_specific_handler 10004028     corelib1:COREDLL.dll
 0002:0000002c       __imp___security_gen_cookie2 1000402c     corelib1:COREDLL.dll
 0002:00000030       __imp_free                 10004030     corelib1:COREDLL.dll
 0002:00000034       __imp_realloc              10004034     corelib1:COREDLL.dll
 0002:00000038       __imp_malloc               10004038     corelib1:COREDLL.dll
 0002:0000003c       __imp__msize               1000403c     corelib1:COREDLL.dll
 0002:00000040       __imp_TerminateProcess     10004040     coredll:COREDLL.dll
 0002:00000044       \177COREDLL_NULL_THUNK_DATA 10004044     coredll:COREDLL.dll
 0002:00000048       dpCurSettings              10004048     DebugZones.obj
 0002:00000490       __security_cookie          10004490     corelib0:seccinit.obj
 0002:00000494       __security_cookie_complement 10004494     corelib0:seccinit.obj
 0002:0000143c       _exitflag                  1000543c     corelib0:cexit.obj
 0002:00001440       __onexitend                10005440     <common>
 0002:00001444       __onexitbegin              10005444     <common>
 0002:00001448       _pRawDllMain               10005448     <common>

 entry point at        0001:00002580

 Static symbols

 0001:00001578       ?CallDriver@@YAHHPAUGPIO_CONFIG@@@Z 10002578 f   gpiosdk.obj
 0001:00001910       ?CallDriver@@YAHHPAUGPIO@@@Z 10002910 f   gpiosdk.obj
 0001:0000219c       ?CallDriver@@YAHHPAUGPIO_EVENT@@@Z 1000319c f   gpiosdk.obj
 0001:000025d0       _DllMainCRTStartupHelper   100035d0 f   corelib0:pegdmain.obj
 0001:000027d0       doexit                     100037d0 f   corelib0:cexit.obj
